:1000000010308A00002800000A108A100A118207A6
:1000100028340C34013406340A108A100A1182077D
:100020008A343834B9342F3488345C3495342F34DE
:1000300044344F344D3441340034003400340034FF
:100040008A3437349F347534883459342934EC3445
:1000500047344334313436344A344D344834003430
:100060008A3437349D3464348834593426345634D1
:100070004734433431343634463438345934003418
:100080008A3438345834AC34883460341A34B03458
:10009000473443342D342D342D342D342D34003455
:1000A0000A108A100A118207483445342534323444
:1000B0002E343034673468342A3441345A34253489
:1000C00032342E343034673468342A340034C33048
:1000D0008400000803197B280130F800F701F70BB2
:1000E0006F28F80B6E284A30F700F70B75280000D0
:1000F0000000800B6C28003406080F398316CA00F4
:10010000490EF700F030F7057708F0394A048312FA
:1001100086000615831606112130F700F70B8E288E
:100120008312061183160611831200348316C70842
:10013000031D9E2883128610A0288316831286141E
:1001400083168610C80E4808C90083127C208316C7
:10015000C80E4808C90083127C204230F700F70B14
:10016000AF280000003414308316C30083126720C8
:100170000F3083168605831286108316861083122D
:100180000611831606118312B3013308023C031CC7
:10019000D52802308316C3008312672003308316EC
:1001A000C90083127C20B30AC5280D30F700F70B75
:1001B000D72802308316C90083127C200D30F70047
:1001C000F70BE028B3013308023C031CF92833087D
:1001D0000420B4008316C701831234088316C800B4
:1001E0008312962002308316C30083126720B30A5D
:1001F000E3288A110A165528013083164402FC3E72
:1002000003181529043E831221298316C5011529D7
:1002100040308316C500152914308316C5001529F2
:1002200054308316C5001529831601304302C507D3
:1002300045088038C600C7014608C80083129620CA
:1002400000340A148A100A118207052908290C298A
:100250001029831642080C3A831203193929063AE9
:1002600003194529073A03194D29053A0319542959
:100270005B298316C7010130C80083129620023023
:100280008316C30083126720692901308316C300D7
:100290000230C4008312FC20692901308316C30098
:1002A000C4008312FC2069298316C7011030C800DE
:1002B000831296206929831642081F3C031C622979
:1002C0000730C2050130C7004208C80083129620DB
:1002D000692900340830F7002017200883168700AA
:1002E0008312071F7529831670298316B301F71728
:1002F0008929F713892903108312071B0314831616
:10030000B30C771789297713F70B7B293308F8008B
:1003100094293F30F71B1130F800F80B8D29F71B9B
:100320007929771B83297B2983120034831642089D
:100330000319072ACA0046080319072ACA0703181F
:10034000A8297F30CA02031C072A0319072AAC29EF
:100350008130CA070318072A4A08F700F801F90193
:10036000FA014308CE00CE174408CD004508CC0062
:100370001830CA00CB014C1CD5294908FA07031CC8
:10038000C729F90A031DC729F80A0319CB1748081A
:10039000F907031CCE29F80A0319CB174708C40034
:1003A000C4174408F8070318CB17CB0DF80CF90C49
:1003B000FA0CCE0CCD0CCC0C0310CA0BBA290130B0
:1003C000F7070318072AF81BEC29CE0DFA0DF90DD3
:1003D000F80DF7030319072ACE1FFD29FA0A031D9A
:1003E000FD29F90A031DFD29F80A031DFD29F80C52
:1003F000F90CFA0CF70A0319072A4308CB0047083F
:10040000CB06CB1F052AF8170B2AF8130B2AF70186
:10041000F801F901FA010000831200348E30F70070
:1004200083164608F8004508F900FA01F808031D8C
:10043000232A7908F800F9010830F702F808031DAB
:10044000232AF7012B2A0310F81B2A2AF90DF80D8D
:10045000F703232AF8130000831200348030831C32
:10046000342A8316CE0683128316D301D4014A0898
:10047000D2004E08D206490803191F2BD100F700FD
:100480004D080319282BD1020319C52A031C842AFD
:100490004E08D700D7174F08D6005008D500D40112
:1004A0000310D70CD60CD50CD40CD10B4F2AD21F6D
:1004B0005C2A53143C2B531051105316CC3084003B
:1004C000512B5312D21B6E2A511C792AD70CD60CF1
:1004D000D50CD40CF70A0319372B792AD71B7C2AA1
:1004E0000310D40DD50DD60DD70DF7030319372BF7
:1004F0006E2A5317E42A53134A08D200CA1F822ACD
:10050000D717302BD713302B4D08D100F7004908EF
:10051000D1024A08D700D7174B08D6004C08D5009F
:10052000D4010310D70CD60CD50CD40CD10B902AC7
:10053000D21F9D2AD3143C2BD3105110D316D03088
:100540008400512BD312D21BAF2A511CBA2AD70CCC
:10055000D60CD50CD40CF70A0319372BBA2AD71BA3
:10056000BD2A0310D40DD50DD60DD70DF7030319F1
:10057000372BAF2AD317E42AD3134E08D200CE1F4D
:10058000C32AD717302BD713302B4E08D700D717D5
:100590004F08D6005008D500D21FD22AD7135315C2
:1005A0003C2B5311D4015110CC308400512BD21B61
:1005B000FA2A4A08D200511CE42AD70CD60CD50CD2
:1005C000D40CF70A0319372BD41FF52AD50A031DBB
:1005D000F52AD60A031DF52AD70A031DF52AD70CDA
:1005E000D60CD50CF70A0319372B531B7B2AD31BC8
:1005F000BC2A192B8030D706D71F022B3C2B4E0864
:10060000D2000F2B4A08D200D708031D0F2BD608A3
:10061000031D0F2BD508031D0F2BF701302BD71B04
:10062000192B0310D40DD50DD60DD70DF70B0F2BAD
:10063000372BD21F1D2BD717302BD713302B4D083C
:10064000F7004E08D7004F08D6005008D500302BD1
:100650004908F7004A08D7004B08D6004C08D500D7
:100660005708F8005608F9005508FA006F2BF701F3
:10067000F801F901FA016F2BD401D509D609D70980
:10068000D409D40A031D4A2BD50A031D4A2BD60AC6
:100690000319D70A53185B2AD3189C2A5319D12A55
:1006A000FF2A0008D507031C5B2BD60A031D5B2B12
:1006B000D70A0319511484030008D607031C632BBF
:1006C000D70A0319511484030008801F803AD70702
:1006D00003185114531A612AD31AA22AD72A0000E8
:1006E00083120034831642080319382CCE004608C2
:1006F0000319382CCE02031C822B7F30CE0703183F
:10070000382C882B8130CE02031C382C0319382C4E
:100710004E08F700F801F901FA01CD014308CC00B9
:10072000CC174408CB004508CA001930CE00490850
:10073000CA020318AB2B0130CB020318AB2BCC023F
:100740000318AB2BCD020318AB2BCD0ACC0ACB0A76
:100750004908CA07DD2B4808CB020318C62B013015
:10076000CC020318C62BCD020318C62BCD0ACC0A27
:100770004808CB074908CA07031CDD2BCB0A031D19
:10078000DD2BCC0A031DDD2BCD0ADD2B470880387D
:10079000CC020318DC2B0130CD020318DC2BCD0A70
:1007A00047088038CC074808CB07031CBA2BCC0A73
:1007B000031DBA2BCD0ABA2B7A14CE0BE02BEB2BF0
:1007C0000310CA0DCB0DCC0DCD0D0310FA0DF90D94
:1007D000F80DCF0D972B4F1CF32B0310F80CF90CD1
:1007E000FA0CCF0CF62BF7030319382CCF1B1F2C58
:1007F0000310CA0DCB0DCC0DCD0D4908CA0203184C
:100800000B2C0130CB0203180B2CCC0203180B2C41
:10081000CD02031C2E2C4808CB020318162C0130E5
:10082000CC020318162CCD02031C2E2C470880384E
:10083000CC0203181F2C0130CD02031C2E2CFA0A07
:10084000031D2E2CF90A031D2E2CF80A031D2E2C35
:10085000F70A0319382CF80CF90CFA0C4308CE00EF
:100860004708CE06CE1F362CF8173C2CF8133C2C2C
:10087000F701F801F901FA010000831200347F301A
:100880008316B500B601B701B801B901BA01BB01C1
:10089000BC01BD01BE01C001B308031D542CF7010A
:1008A000F801F901FA018C2D4008C00A33078400D1
:1008B0000008BF003F082F3C0318622C3F08393C5A
:1008C00003186E2C3F082B3C03196E2C3F082D3C5F
:1008D00003196E2C3F082E3C031D582D3F082D3C5C
:1008E000031D7A2C0130BD004008C00A3307840084
:1008F0000008BF003F082F3C0318E12C3F08393C9B
:10090000031CE12CBE08031DE12CC501C4012030ED
:10091000C3008230C2003C08C9003B08C8003A0846
:10092000C7003908C6008312962177088316C100D4
:100930007808C2007908C3007A08C400C6013F08DD
:10094000C50083120E22831083164408CC0043088E
:10095000CB004208CA004108C9007A08D0007908D3
:10096000CF007808CE007708CD0083122E227708BA
:100970008316C5007808C6007908C7007A08C80041
:1009800083144808CC004708CB004608CA00450835
:10099000C900D001CF014030CE008430CD00831299
:1009A0002E227A088316BC007908BB007808BA00AA
:1009B0007708B9004008C00A330784000008BF0068
:1009C0007A2C3F082E3C031DED2C0130BE00400860
:1009D000C00A330784000008BF003F082F3C0318FB
:1009E0004D2D3F08393C031C4D2D3E0B4D2D380835
:1009F000C5003708C4003608C3003508C200C90165
:100A0000C8012030C7008230C600831296217A08C0
:100A10008316B8007908B7007808B6007708B500E3
:100A200030303F02C601C50083120E227A088316B9
:100A3000C5007908C4007808C3007708C2003808E8
:100A4000C9003708C8003608C7003508C600831239
:100A50007223831083163C08CC003B08CB003A0875
:100A6000CA003908C9007A08D0007908CF00780890
:100A7000CE007708CD0083122E227A088316BC00A0
:100A80007908BB007808BA007708B9004008C00AA6
:100A9000330784000008BF00ED2C3F082B3C031DEA
:100AA000572D4008C00A330784000008BF005A2CA5
:100AB0003D0B732DC501C4018030C3007F30C200DF
:100AC0003C08C9003B08C8003A08C7003908C600FE
:100AD000831296217A088316BC007908BB00780837
:100AE000BA007708B900B4080319842DC0080319A7
:100AF000802DC00334088400400833078000842D13
:100B000034088400330880003908F7003A08F800F8
:100B10003B08F9003C08FA008312003483164208AF
:100B2000B63CC200FA014308C600C3170310C30C49
:100B3000C40CC50CFA0CF90CF80CF70CC20B962D72
:100B4000C61FAD2DF709F809F909FA09F70A0319C3
:100B5000F80A0319F90A0319FA0A83128A110A1208
:100B6000442EF701F801F901FA018316CA01CB01FD
:100B7000CC01CD0149084804470446040319F02D6F
:100B80002030CE000310C20DC30DC40DC50DCA0D1B
:100B9000CB0DCC0DCD0D49084D02031DD92D4808B4
:100BA0004C02031DD92D47084B02031DD92D4608C1
:100BB0004A02031CEA2D4608CA024708031C470FD5
:100BC000CB024808031C480FCC024908031C490FFC
:100BD000CD020314F70DF80DF90DFA0DCE0BC22D51
:100BE0000000CA3084008312003404088316BC005D
:100BF0003B08BD000319172E3A08C5003908C40088
:100C00003808C3003708C200C901C8012030C70036
:100C10008230C600831296217A088316BA007908BA
:100C2000B9007808B8007708B700BD0BFC2D7E30FE
:100C3000F700F801B81BF817F901FA0183103A0818
:100C4000CC003908CB003808CA003708C9007A0838
:100C5000D0007908CF007808CE007708CD00831245
:100C60002E227A088316BA007908B9007808B800ED
:100C70007708B7003A08C5003908C4003808C3002F
:100C80003708C20083128E2D7A088316BA007908BD
:100C9000B9007808B8007708B700BA1F5C2EBC030B
:100CA000BC16B709B809B909BA09B70A0319B80ACD
:100CB0000319B90A0319BA0A3B30C1009A30C000BF
:100CC000CA30BF00BE010A30BD003B080319BC0A90
:100CD0003A08C5003908C4003808C3003708C20004
:100CE0004108C9004008C8003F08C7003E08C600C8
:100CF0008312B12500088316B700840A0008B800E3
:100D0000840A0008B900840A0008BA00FD3084078C
:100D1000F708031D9E2E3B0A3D0203199E2E3C0838
:100D20000319A02E0F393D020319982E0318D82E4F
:100D3000BC1BD82E3C1BA02E2030D22E2030BC0550
:100D4000BC1EB02EBC123B08031DBC037708BC00C0
:100D50002D30C2008312292183163C08F700BC0104
:100D60003B083D02031DC02E7708BC002E30C20098
:100D70008312292183163C08F7002030BC0500307F
:100D80003030BC1ED22EBC123B08031DBC037708BA
:100D9000BC002D30C2008312292183163C08F700C5
:100DA000BC013030F7077708C2008312292183166F
:100DB0004108C5004008C4003F08C3003E08C20007
:100DC000C901C801C7010A30C6008312B1257A08DB
:100DD0008316C1007908C0007808BF007708BE00FC
:100DE000BD0B682E8312003483163308B600B50895
:100DF00003190D2F34088400800803190D2F3608BD
:100E0000B60AB7003408B40A84000008B8003708EE
:100E1000840038088000B503F72EB5080319162F93
:100E20003608B60A84008001B5030D2F3308F80098
:100E30008312003483166408E6006308E70065083F
:100E4000003C03182F2F6708840066080002031D6A
:100E50002C2F6708F800312FE70AE5031F2F003019
:100E6000F8008312003410308316E700F701FA010E
:100E7000E40CE30C031C422F6508F7070318FA0A79
:100E80006608FA07FA0CF70CF90CF80CE70B382F88
:100E900083128A110A16262B5308DA005708DA063D
:100EA000DA1F572F03110310D31B03148A2F530883
:100EB000DA005608DB005208DB020319652FDA1F3F
:100EC0008A2F0308013A83008A2F5708DB00530852
:100ED000DB020319712FDA1F8A2F0308013A8300FE
:100EE0008A2F5808DB005408DB0203197D2FDA1F14
:100EF0008A2F0308013A83008A2F5908DB0055081E
:100F0000DB020319892FDA1F8A2F0308013A8300B5
:060F10008A2F03100034DB
:101000003E08D5003D08D4003C08D3003B08D20080
:10101000D901D801D701D6018A114C278A150318A6
:101020001328031D1828F701F801F901FA01A9286E
:101030003E08C2003D08C1003C08C0003B08BF009C
:101040003F30C7004708C800470884000008CA01AD
:10105000C9007F304907CB004A08CC000318CC0AEE
:1010600003104C0CFA004B0CF900CD00480884002A
:101070004D0880004208C6004108C5004008C40071
:101080003F08C3003E088316C50083123D0883163F
:10109000C40083123C088316C30083123B088316E6
:1010A000C200831242088316C900831241088316C6
:1010B000C800831240088316C70083123F088316B6
:1010C000C6008A11831272238A1583104208831680
:1010D000CC00831241088316CB008312400883168C
:1010E000CA0083123F088316C9007A08D000790825
:1010F000CF007808CE007708CD008A1183122E2207
:101100008A157A08C2007908C1007808C0007708FB
:10111000BF004708840080034608D5004508D40076
:101120004408D3004308D2004208D9004108D8003F
:101130004008D7003F08D6008A114C278A15031DA6
:101140003A284308F7004408F8004508F900460823
:10115000FA008A110A16E12C5110D1104408C80077
:101160004308C7004208C6004108C5004408D5002E
:101170004308D4004208D3004108D200D901D80165
:10118000D701D6018A114C278A15031CCA2851148D
:101190008030C606D501D401D3017F30D200480883
:1011A000D9004708D8004608D7004508D6008A115C
:1011B0004C278A15031CFF288316C501C401C301EF
:1011C0007F30C200831248088316C9008312470883
:1011D0008316C800831246088316C7008312450889
:1011E0008316C6008A11831272238A157A08C800F2
:1011F0007908C7007808C6007708C500D1140A30FE
:101200008316C5008930C4003430C3007C30C2006E
:10121000831248088316C900831247088316C80042
:10122000831246088316C700831245088316C6003A
:101230008A11831296218A157708D2007808D30084
:101240007908D4007A08D5008316C500831279087E
:101250008316C400831278088316C30083127708AC
:101260008316C200831248088316C90083124708F8
:101270008316C800831246088316C70083124508E8
:101280008316C6008A11831296218A157708D60024
:101290007808D7007908D8007A08D90083107A082E
:1012A0008316CC00831279088316CB00831278084A
:1012B0008316CA00831277088316C9007C30D000D9
:1012C0007930CF003530CE008130CD008A118312C5
:1012D0002E228A157A08CC007908CB007808CA003B
:1012E0007708C9004C088316C50083124B08831683
:1012F000C40083124A088316C30083124908831668
:10130000C200831248088316C90083124708831657
:10131000C800831246088316C70083124508831647
:10132000C6008A11831296218A157708D2007808A0
:10133000D3007908D4007A08D5008316C50083123B
:1013400079088316C400831278088316C3008312B9
:1013500077088316C200831248088316C9008312D7
:1013600047088316C800831246088316C7008312F5
:1013700045088316C6008A11831296218A157708BC
:10138000D6007808D7007908D8007A08D9008310E9
:101390007A088316CC00831279088316CB00831257
:1013A00078088316CA00831277088316C9003F3075
:1013B000D0000230CF003330CE008330CD008A1110
:1013C00083122E228A157A08CC007908CB0078087F
:1013D000CA007708C9004C088316C50083124B0861
:1013E0008316C40083124A088316C3008312490877
:1013F0008316C200831248088316C9008312470867
:101400008316C800831246088316C7008312450856
:101410008316C6008A11831296218A157708D20096
:101420007808D3007908D4007A08D5008316C5005F
:10143000831279088316C400831278088316C300C8
:10144000831277088316C200831248088316C900E6
:10145000831247088316C800831246088316C70004
:10146000831245088316C6008A11831296218A15B5
:101470007708D6007808D7007908D8007A08D9000C
:1014800083107A088316CC00831279088316CB0068
:10149000831278088316CA00831277088316C9005E
:1014A0003330D0008C30CF001E30CE008330CD00E2
:1014B0008A1183122E228A157A08CC007908CB0073
:1014C0007808CA007708C9008316C501C401C301A2
:1014D0007F30C200831248088316C9008312470870
:1014E0008316C800831246088316C7008312450876
:1014F0008316C6008A11831296218A157708D200B6
:101500007808D3007908D4007A08D5008316C5007E
:10151000831279088316C400831278088316C300E7
:10152000831277088316C200831248088316C90005
:10153000831247088316C800831246088316C70023
:10154000831245088316C6008A11831296218A15D4
:101550007708D6007808D7007908D8007A08D9002B
:1015600083107A088316CC00831279088316CB0087
:10157000831278088316CA00831277088316C9007D
:101580001B30D000E430CF003530CE008230CD00AB
:101590008A1183122E228A157A08D0007908CF008A
:1015A0007808CE007708CD0050088316C500831256
:1015B0004F088316C40083124E088316C30083129B
:1015C0004D088316C200831248088316C90083128F
:1015D00047088316C800831246088316C700831283
:1015E00045088316C6008A11831296218A1577084A
:1015F000D2007808D3007908D4007A08D500831681
:10160000C500831279088316C400831278088316F4
:10161000C300831277088316C2008312480883161A
:10162000C900831247088316C80083124608831630
:10163000C700831245088316C6008A1183129621BB
:101640008A157708D6007808D7007908D8007A0874
:10165000D90083107A088316CC0083127908831688
:10166000CB00831278088316CA008312770883168A
:10167000C900A430D000DB30CF006730CE0083300B
:10168000CD008A1183122E228A157A08D00079089B
:10169000CF007808CE007708CD0050088316C5002B
:1016A00083124F088316C40083124E088316C300AA
:1016B00083124D088316C200831248088316C9009E
:1016C000831247088316C800831246088316C70092
:1016D000831245088316C6008A11831296218A1543
:1016E0007708D2007808D3007908D4007A08D500AA
:1016F0008316C500831279088316C4008312780804
:101700008316C300831277088316C2008312480829
:101710008316C900831247088316C800831246083F
:101720008316C700831245088316C6008A118312E8
:1017300096218A157708D6007808D7007908D8004E
:101740007A08D90083107A088316CC0083127908AE
:101750008316CB00831278088316CA008312770899
:101760008316C9003330D0008C30CF001E30CE003D
:101770008330CD008A1183122E228A157A08D00078
:101780007908CF007808CE007708CD004808831686
:10179000C500831247088316C400831246088316C7
:1017A000C300831245088316C20083124C088316B7
:1017B000C90083124B088316C80083124A08831697
:1017C000C700831249088316C6008A118312962126
:1017D0008A157708D2007808D3007908D4007A08EF
:1017E000D5008316C500831279088316C4008312BE
:1017F00078088316C300831277088316C200831209
:1018000050088316C90083124F088316C80083123C
:101810004E088316C70083124D088316C6008A112E
:10182000831272238A157A08CC007908CB007808D5
:10183000CA007708C900D11C432C8314DB308316FF
:10184000CC000F30CB004930CA007F30C900831272
:101850004C088316D00083124B088316CF008312E6
:101860004A088316CE00831249088316CD008A11D8
:1018700083122E228A157A08CC007908CB007808CA
:10188000CA007708C900511C472C8030CA06490895
:10189000F7004A08F8004B08F9004C08FA00003439
:1018A0003F10C0013608D5003508D4003408D300F5
:1018B0003308D200D901D801D701D6018A114C27AB
:1018C0008A150318652C031D7C2C3A08D5003908AD
:1018D000D4003808D3003708D200D901D801D70185
:1018E000D6018A114C278A150318782C031D7A2CEF
:1018F00003307B2C0430902C3A08D5003908D400F2
:101900003808D3003708D200D901D801D701D60151
:101910008A114C278A15031C8F2C0230902C013021
:10192000C0003608D5003508D4003408D300330889
:10193000D200D901D801D701D6018A114C278A15C6
:10194000031CA52C3F148030B4063A08D500390892
:10195000D4003808D3003708D200D901D801D70104
:10196000D6018A114C278A15031CB82C8030B80682
:101970003A08D5003908D4003808D3003708D20017
:10198000D901D801D701D6018A114C278A15031D28
:10199000F02C3608D5003508D4003408D3003308BD
:1019A000D200D901D801D701D6018A114C278A1556
:1019B0000319EF2C3F1CE62C7F30F700C930F800EC
:1019C0000F30F900DB30FA00922DEF2C7F30F7005A
:1019D0004930F8000F30F900DB30FA00922D922DDB
:1019E00036088316C500831235088316C400831297
:1019F00034088316C300831233088316C20083128F
:101A00003A088316C900831239088316C800831266
:101A100038088316C700831237088316C6008A1158
:101A2000831272238A157A08BE007908BD007808EF
:101A3000BC007708BB0001304002FC3E0318922D29
:101A4000043E952D3E08C4003D08C3003C08C2007A
:101A50003B08C100AC20922D922D3E08C4003D08E9
:101A6000C3003C08C2003B08C100AC200408C10010
:101A70008314DB308316CC000F30CB004930CA0012
:101A80008030C9007A08D0007908CF007808CE00ED
:101A90007708CD008A1183122E228A15410884000E
:101AA000922D922D3E08C4003D08C3003C08C200A0
:101AB0003B08C100AC207708C1007808C200790853
:101AC000C3007A08C4000408C500831444088316C0
:101AD000CC00831243088316CB008312420883167E
:101AE000CA00831241088316C900DB30D0000F30D2
:101AF000CF004930CE008030CD008A1183122E22D3
:101B00008A1545088400922D922D3E08C4003D0898
:101B1000C3003C08C2003B08C100AC208030F8067E
:101B2000922D922D8A110A16432D0A148A100A1535
:0A1B30008207222D2D2D522D852D48
:10200000A701A60184011F308305831605108312E2
:102010000514831605108312051483161F149F14CC
:102020001F159F1107309C00FF308312A000A101F3
:102030000130A200A301A401A50183161F149F145F
:102040001F159F1183121F109412A01220088316CF
:102050008700831220162008831687008312A011A0
:1020600020088316870000308312940083169400A2
:102070000108C73908388100831290010030F80048
:10208000920000308316920007309C000508033050
:10209000F700F70B49281C0883120D13FE30831636
:1020A0009D0005150A128312B3280A16B20A3208D7
:1020B000033C031CB201C8308316C3000A1283120A
:1020C00067200A1601308316C3000230C4000A12CA
:1020D0008312FC200A16320EF700F030F70577085D
:1020E000083EB400B50035080A120C200A16003864
:1020F00003198228B50A8316C2000A128312292105
:102100000A167328EE010A126A210A167808243C7E
:10211000031D8328F00170083A3C031CA4280A120E
:102120006A210A167808F10071082A3C031D9D28CF
:102130003330700784008001A42833307007840096
:1021400071088000F00A8B280C308316C30004301D
:10215000C4000A128312FC200A1639308316B30019
:102160006F30B4000A1283123F240A167708F20077
:102170007808F3007908F4007A08F500440883161B
:10218000C2000A12831229210A1620308316C200C7
:102190000A12831229210A16453084007508831615
:1021A000BA007408B9007308B8007208B700BB0120
:1021B0000A128312F5250A1620308316C2000A126D
:1021C000831229210A1601308316C3000330C4008C
:1021D0000A128312FC200A16A0308316B300463080
:1021E000B4000930B5000A128312F4260A168316C9
:1021F000A901A03084000030000403190C29040850
:10220000F2000008C2000A12831229210A1672087D
:102210008400840A8316FB282A30C2000A12831223
:1022200029210A16A0308316B3005330B4000930B8
:10223000B5000A128312F4260A168316A901A030EB
:10224000840000300004031932290408F200000859
:10225000C2000A12831229210A1672088400840A15
:10226000831621292A30C2000A12831229210A1654
:1022700048308316B3006F30B4000A1283123F2433
:102280000A167A08AB007908AA007808A90077082E
:10229000A800C80146308316B3006F30B4000A129C
:1022A00083123F240A168316C501C4017030C3008F
:1022B0008430C2007A08C9007908C8007808C700CD
:1022C0007708C6000A12831296210A160408F20043
:1022D00083102B088316CC0083122A088316CB00A8
:1022E000831229088316CA00831228088316C9009E
:1022F0007A08D0007908CF007808CE007708CD00A2
:102300000A1283122E220A16720884007A08AB0081
:102310007908AA007808A9007708A8005530831624
:10232000B3006F30B4000A1283123F240A167A08F1
:10233000AF007908AE007808AD007708AC00D50191
:1023400053308316B3006F30B4000A1283123F2457
:102350000A168316C501C4017030C3008430C20060
:102360007A08C9007908C8007808C7007708C6004D
:102370000A12831296210A160408F20083102F080D
:102380008316CC0083122E088316CB0083122D08EF
:102390008316CA0083122C088316C9007A08D0005D
:1023A0007908CF007808CE007708CD000A12831292
:1023B0002E220A16720884007A08AF007908AE004F
:1023C0007808AD007708AC0061308316B3006F3039
:1023D000B4000A1283123F240A1601306F07F2007C
:1023E00072088316B4006F30B5000A30B600BA0127
:1023F000BB013030BD003130BE003230BF00333061
:10240000C0003430C1003530C2003630C300373030
:10241000C4003830C5003930C6006130C7006230B2
:10242000C8006330C9006430CA006530CB00663034
:10243000CC006730CD006830CE006930CF006A3004
:10244000D0006B30D1006C30D2006D30D3006E30D4
:10245000D4006F30D5007030D6007130D7007330A3
:10246000D8007430D9007530DA007630DB00773070
:10247000DC007830DD007930DE007A30DF00E0010A
:102480003408B700370884000008203C031D4A2A9E
:10249000B70A422A3708840000082D3C0319562A3F
:1024A0003708840000082B3C031D5B2A3708B70A55
:1024B000840000085C2A2B30BC003C082D3C031D26
:1024C0006C2AB5080319682A35088400340880008E
:1024D0000030F800F900722BB61B772A360B712AF0
:1024E000772AB61B832A3608243C0318832AB508AA
:1024F00003197E2A35088400340880000030F80073
:10250000F900722BE92AB6080319C02A3608103CD4
:10251000031DA02A370884000008303C031DA02AB0
:102520000130370784000008783C03199E2A0130E7
:10253000370784000008583C031DA02A0230B70763
:102540003608083C031DAC2A370884000008303CDC
:10255000031DAC2A0130B7073608023C031DBF2A11
:10256000370884000008303C031DBF2A01303707BC
:1025700084000008623C031DBF2A0230B707E92A25
:10258000370884000008303C0319C92A0A30B60015
:10259000E92A0130370784000008783C0319D72A5C
:1025A0000130370784000008583C031DDC2A103036
:1025B000B6000230B707E92A013037078400000867
:1025C000623C031DE72A0230B600B707E92A08304B
:1025D000B6003708B800370884000008303C031DF7
:1025E000F32AB70AEB2A370884000008E100403CD0
:1025F0000318012B61085A3C031C012B6108203889
:10260000022B6108E200BD30E3006108E4003608F7
:10261000E5000A1283121A270A1678088316B900F1
:10262000B9080319582BFA013608F700B61BFA034C
:10263000E1007A08E2003B08E4003A08E30062089F
:10264000E6006108E5000A128312332F0A167908A2
:102650008316E3007808E200BD303902FA01620710
:10266000F80063080318630FFA077808BA007A08BD
:10267000BB00B70A370884000008E100403C03189B
:10268000482B61085A3C031C482B61082038492B11
:102690006108E200BD30E3006108E4003608E500AF
:1026A0000A1283121A270A1678088316B900102B0B
:1026B00037083802031D672BB5080319632B35084B
:1026C0008400340880000030F800F900722BB5084F
:1026D00003196E2B35088400370880003A08F8008B
:1026E0003B08F90079088312B1007808B000320E77
:1026F000F700F030F7057708043EB4000330B40764
:1027000034080A120C200A16FA00B40334080A121C
:102710000C200A16F900B40334080A120C200A1619
:10272000F80034030A120C200A16F700B5007808E6
:10273000B6007908B7007A08B80083143808831601
:10274000CC00831237088316CB0083123608831619
:10275000CA00831235088316C90083122F08831616
:10276000D00083122E088316CF0083122D08831603
:10277000CE0083122C088316CD000A1283122E225B
:102780000A167708B9007808BA007908BB007A08F9
:10279000BC008316C50083123B088316C400831255
:1027A0003A088316C300831239088316C200C90190
:1027B000C030C8001730C7008930C6000A12831223
:1027C00096210A167A08AF007908AE007808AD00A5
:1027D0007708AC00320EF700F030F7057708B40048
:1027E0000330B40734080A120C200A16FA00B403A6
:1027F00034080A120C200A16F900B40334080A122D
:102800000C200A16F80034030A120C200A16F700EE
:10281000B5007808B6007908B7007A08B8008314C4
:1028200038088316CC00831237088316CB00831236
:1028300036088316CA00831235088316C90083122E
:102840002B088316D00083122A088316CF00831228
:1028500029088316CE00831228088316CD000A1299
:1028600083122E220A167708B9007808BA00790870
:10287000BB007A08BC008316C50083123B08831690
:10288000C40083123A088316C300831239088316E2
:10289000C200C901C030C8006730C7008930C60017
:1028A0000A12831296210A167A08AB007908AA0048
:1028B0007808A9007708A80001308316C300043007
:1028C000C4000A128312FC200A162F088316C500C2
:1028D00083122E088316C40083122D088316C300AA
:1028E00083122C088316C20083122F088316C90096
:1028F00083122E088316C80083122D088316C70082
:1029000083122C088316C6000A12831296210A1617
:102910007708B3007808B4007908B5007A08B600E3
:102920002B088316C50083122A088316C40083125D
:1029300029088316C300831228088316C200831255
:102940002B088316C90083122A088316C800831235
:1029500029088316C700831228088316C6000A12A6
:10296000831296210A16831036088316CC00831230
:1029700035088316CB00831234088316CA008312ED
:1029800033088316C9007A08D0007908CF00780888
:10299000CE007708CD000A1283122E220A1677087D
:1029A000B7007808B8007908B9007A08BA00BE0004
:1029B0003908BD003808BC003708BB000A128A1568
:1029C00000280A168A117708B8007808B900790833
:1029D000BA007A08BB00893084003B088316BA002D
:1029E00083123A088316B900831239088316B80097
:1029F000831238088316B700BB010A128312F5252B
:102A00000A166D308316C2000A12831229210A1693
:102A100020308316C2000A12831229210A160130BF
:102A20008316C300C4000A128312FC200A162F0862
:102A3000D5002E08D4002D08D3002C08D200D901CF
:102A4000D801D701D6010A124C270A16031D302DD2
:102A50006F30AF001230AE000330AD007530AC0007
:102A60002B08B6002A08B5002908B4002808B300CE
:102A70002F08BA002E08B9002D08B8002C08B7009E
:102A80000A128A15502C0A168A1145308316C50081
:102A90007630C4007430C3007F30C2007A08C900A9
:102AA0007908C8007808C7007708C6000A128312A0
:102AB00096210A160408B30083148316CC01CB01B7
:102AC0004030CA008030C9007A08D0007908CF00B1
:102AD0007808CE007708CD000A1283122E220A163B
:102AE000330884007A08AF007908AE007808AD009A
:102AF0007708AC002F08D5002E08D4002D08D3008D
:102B00002C08D200D901D801D701D6010A124C27CE
:102B10000A16031CAD2D83102F088316CC008312D8
:102B20002E088316CB0083122D088316CA00831249
:102B30002C088316C900D001CF014030CE0082306E
:102B4000CD000A1283122E220A167A08AF007908E5
:102B5000AE007808AD007708AC00D501D401403054
:102B6000D3008230D2002F08D9002E08D8002D08BB
:102B7000D7002C08D6000A124C270A16031CE22D97
:102B800083142F088316CC0083122E088316CB00E3
:102B900083122D088316CA0083122C088316C900DD
:102BA000D001CF014030CE008230CD000A12831216
:102BB0002E220A167A08AF007908AE007808AD0018
:102BC0007708AC0042308316C2000A128312292112
:102BD0000A1645308316C2000A12831229210A16EA
:102BE000013084002F088316BA0083122E08831642
:102BF000B90083122D088316B80083122C0883169F
:102C0000B700BB010A128312F5250A166830831635
:102C1000C2000A12831229210A162A308316C20022
:102C20000A12831229210A1631088316C60083125C
:102C300030088316C5000A1283120E220A16893044
:102C40008316C5008830C4000830C3007A30C20043
:102C50007A08C9007908C8007808C7007708C60054
:102C60000A12831296210A167A08AB007908AA0084
:102C70007808A9007708A80083142F088316CC00D1
:102C800083122E088316CB0083122D088316CA00E8
:102C900083122C088316C90083122B088316D000D8
:102CA00083122A088316CF00831229088316CE00C8
:102CB000831228088316CD000A1283122E220A16C8
:102CC0007A08AF007908AE007808AD007708AC004C
:102CD0002F08D5002E08D4002D08D3002C08D200D0
:102CE000D901D801D701D6010A124C270A16031CB4
:102CF0009B2E83102F088316CC0083122E08831678
:102D0000CB0083122D088316CA0083122C08831669
:102D1000C900D001CF014030CE008230CD000A1270
:102D200083122E220A167A08AF007908AE007808BE
:102D3000AD007708AC00D501D4014030D30082301B
:102D4000D2002F08D9002E08D8002D08D7002C0853
:102D5000D6000A124C270A16031CD02E83142F0803
:102D60008316CC0083122E088316CB0083122D0805
:102D70008316CA0083122C088316C900D001CF0124
:102D80004030CE008230CD000A1283122E220A1665
:102D90007A08AF007908AE007808AD007708AC007B
:102DA00048308316C2000A12831229210A164530C0
:102DB0008316C2000A12831229210A1601308400E8
:102DC0002F088316BA0083122E088316B9008312C7
:102DD0002D088316B80083122C088316B700BB0198
:102DE0000A128312F5250A160730B30033080A12B7
:102DF00050200A16B30AF7008316C2000A12831283
:102E000029210A160B303302031DF62E01308400EF
:102E10002B088316BA0083122A088316B90083127E
:102E200029088316B800831228088316B700BB014F
:102E30000A128312F5250A1668308316C2000A1298
:102E4000831229210A162A308316C2000A1283121D
:082E500029210A168228630003
:02400E00393F38
:00000001FF
